:020000040000FA
:04B5000086EF5AF088
:02B50800100031
:10B50C009BEC5EF0ACEC5EF0D38CD38AD3889B8C36
:10B51C00FF0E926EFF0E936EFF0E946E949CB88A83
:10B52C00B88882BE43D293968186040E046E67EC73
:10B53C005EF08196040E046E67EC5EF0FBD960D869
:10B54C001FEE55F0B20EF66EBE0EF76E2FEC5FF0DE
:10B55C00550E2F6F0F0E306F6FEC5EF051D81FEE43
:10B56C0055F0880EF66EBE0EF76E2FEC5FF0550E92
:10B57C002F6F0F0E306F6FEC5EF081868BDADAD99D
:10B58C003FD81FEE55F0DA0EF66EBE0EF76E2FECAE
:10B59C005FF0550E2F6F0F0E306F6FEC5EF030D8E2
:10B5AC001FEE55F0F80EF66EBE0EF76E2FEC5FF038
:10B5BC00550E2F6F0F0E306F6FEC5EF08CEC5EF053
:10B5CC0027C011F03A0E115DD8B4FCD011C005F0B3
:10B5DC00580E096EB7EC5EF000C031F011C005F0EA
:10B5EC00780E096EB7EC5EF031510010336F33A159
:10B5FC0006D011C027F096EC5EF002D8D7D1DED77A
:10B60C000D0E276F96EC5EF00A0E276F96EC5EF02F
:10B61C0012001A6B186B8CEC5EF027C011F011C085
:10B62C0009F0600E056EC5EC5EF000C031F011C083
:10B63C0005F0670E096EC5EC5EF031510014336FE6
:10B64C0033A102D0200E115F300E115DD8B003D0A3
:10B65C00010E1A6F120011514608D8B003D0010E1A
:10B66C001A6F120011C009F0390E056EC5EC5EF0B0
:10B67C0000C031F011C005F0410E096EC5EC5EF052
:10B68C0031510014336F33A103D0010E1A6F120025
:10B69C00300E115D186F410E115DD8A003D0370E1E
:10B6AC00115D186F1200176BB4DF1851100DF3CF2A
:10B6BC0028F01A53D8A404D0ACDF18512825176FE2
:10B6CC0012C028F017512825126F1200300E1825C1
:10B6DC00116F18510908D8B003D0370E1825116F07
:10B6EC0011C027F01DDB12000EC006F00DC005F0D6
:10B6FC00096A100E0A6EEAEC5EF005C018F0E6DF7F
:10B70C0018C005F0066A096A100E0A6E1EEC5FF08E
:10B71C0001C032F000C031F031510D5D296F325152
:10B72C000E592A6F2AC006F029C005F0096A010ECD
:10B73C000A6EEAEC5EF005C018F0C8DF18C005F020
:10B74C00066A096A010E0A6E1EEC5FF001C032F047
:10B75C0000C031F03151295D2B6F32512A592C6FB9
:10B76C002CC006F02BC005F0100E096E0A6A2CDBFB
:10B77C0005C018F0ABDF1851100DF3CF33F0335177
:10B78C002B5D186FA3DF120017C005F0100E096EA9
:10B79C0009DB05C018F09ADF18C028F02851100DED
:10B7AC00F3CF33F03351175D186F90DF1200AEDA20
:10B7BC0027C011F01B0E115DD8B4DFD63A0E115D07
:10B7CC00D8A4F5D78196126B6EDF1A53D8A4B6D0D5
:10B7DC007F0E1715136F2008D8A0BED01353D8B402
:10B7EC0087D061DF1A53D8A4A9D017C01EF05BDF35
:10B7FC001A53D8A4A3D017C01DF055DF1A53D8A4E0
:10B80C009DD0040E175DD8A41AD0020E135DD8A4D7
:10B81C00A3D049DF1A53D8A491D045DF1A53D8A42A
:10B82C008DD017C016F012C037F03DDF371D336FC7
:10B83C003329126F1751125DD8A49CD0B8D7175367
:10B84C00D8A4A6D01653D8A4B2D7010E336F135177
:10B85C003315316F31C005F0010E096E82DA00B07C
:10B86C007BD0106B010E135DD8A00ED0102B1BDFFC
:10B87C000FEE32F01051E926E86AEA2217C0EFFF0A
:10B88C001351105DD8A0F2D712C037F00CDF371D62
:10B89C00336F3329126F1751125DD8A46BD046D871
:10B8AC008186010E106F0FEE32F01051E926E86A16
:10B8BC00EA22EFCF23F00FEE32F01051E924316F72
:10B8CC00E86AEA20326F010E3125E96E000E322152
:10B8DC00EA6EEFCF24F04FD9020E1D27000E1E2367
:10B8EC00020E10271351105DD8A0DDD723D85FD7D7
:10B8FC001DD815C006F014C005F0FF0E096EFF0E22
:10B90C000A6E34DA001E00B0A8D814D8FFD927C0AC
:10B91C0011F00D0E115DD8B430D60A0E115DD8B4ED
:10B92C002CD61B0E115DD8B428D6F0D7130E276F6A
:10B93C00F7D91200110E276FF3D9120061DE1FEE3A
:10B94C0055F0FC0EF66EBE0EF76E83DA550E2F6FA9
:10B95C000F0E306FBED931D053DE1FEE55F00A0EEC
:10B96C00F66EBF0EF76E75DA550E2F6F0F0E306F29
:10B97C00B0D923D045DE1FEE55F01A0EF66EBF0E71
:10B98C00F76E67DA550E2F6F0F0E306FA2D915D0E8
:10B99C0037DE1FEE55F02A0EF66EBF0EF76E59DA33
:10B9AC00550E2F6F0F0E306F94D907D0C80E026E44
:10B9BC00036A79D99B9CF8EF5FF0BCDF21DE1FEEA8
:10B9CC0055F03A0EF66EBF0EF76E43DA550E2F6F2A
:10B9DC000F0E306F7ED99AD927C011F01B0E115D56
:10B9EC00D8A4F9D70DDEC9D5F29E550EA76EAA0EB6
:10B9FC00A76EA6821200010EEA6EE96AF86A15C0FB
:10BA0C0006F014C005F0040E096E0A6ADDD906C0F2
:10BA1C0032F005C031F0FF0E3115336F346B33C08B
:10BA2C0035F0030E1415316F326B32C006F031C095
:10BA3C0005F0400E096E0A6AFBD900C036F035C01D
:10BA4C00F7FF36C0F6FF0F6B0F2B0900F5CFEEFF9B
:10BA5C00400E0F5DD8A0F8D71200F86A35C0F7FF7A
:10BA6C0036C0F6FFA68EA69CA684A688BDDF0A006B
:10BA7C00010EEA6EE96A0F6B0F2BEECFF5FF0F008C
:10BA8C00400E0F5DD8A0F8D7A68EA69CA684ACDF7E
:10BA9C00A69412001D6BB50E1E6F1EC006F01DC0C5
:10BAAC0005F0400E096E0A6A8FD906C015F005C064
:10BABC0014F0A1DF010EEA6EE96AEECF38F0EECF9A
:10BACC0039F0EECF3BF0EECF3CF0146B156B93DFFF
:10BADC00010EEA6EE96AEECF3EF0EECF3FF0EECF0C
:10BAEC0041F0EECF42F039C006F038C005F03FC04F
:10BAFC000AF03EC009F03AD9001E00C031F03CC03B
:10BB0C0006F03BC005F042C00AF041C009F02ED946
:10BB1C00001E31510010336F33A127D01D6B1E6BEB
:10BB2C0039C024F038C023F05AD8020E1D6F1E6B9A
:10BB3C003CC024F03BC023F052D88FDFFF0E146FB3
:10BB4C00020E156F58DFF40E1D6FBF0E1E6F010E27
:10BB5C00236FEF0E246F43D8F60E1D6FBF0E1E6FB2
:10BB6C00236BF00E246F3BD878DF166BFF0E146F2F
:10BB7C00FF0E156F12001EC01FF0206B206B20C033
:10BB8C0006F01FC005F0B50E096E0A6AFDD8001E3E
:10BB9C0000B05DD01EC020F01DC01FF01EC006F00E
:10BBAC001DC005F0096A0A6AE1D800A004D0F00EA5
:10BBBC001D6FBF0E1E6F1EC006F01DC005F0020EDD
:10BBCC00096E0A6AD3D800A004D0F20E1D6FBF0E06
:10BBDC001E6F05D820C01EF01FC01DF012001EC025
:10BBEC0006F01DC005F0400E096E0A6AEDD806C0BD
:10BBFC001CF005C01BF01CC006F01BC005F015C0E6
:10BC0C000AF014C009F0B2D8001E00A014D015C060
:10BC1C0006F014C005F0FF0E096EFF0E0A6EA6D8D2
:10BC2C00001E00B01ADF1CC015F01BC014F0E3DEC0
:10BC3C002E0E276F75D8010EEA6E3F0E1D15316F53
:10BC4C0031C0E9FF23C0EEFF24C0EEFF1200819645
:10BC5C00D7DC1FEE55F0520EF66EBF0EF76EF9D80C
:10BC6C00550E2F6F0F0E306F34D81EC00EF01DC046
:10BC7C000DF03ADD1FEE55F0640EF66EBF0EF76E4A
:10BC8C00E8D8550E2F6F0F0E306F23D806EC5BF0F3
:10BC9C0051DE3CD827C011F01B0E115DD8A4F9D78A
:10BCAC00FF000300FFD7032A040E016EA50E006EE1
:10BCBC00002EFED7012EFAD7022EF6D7032EF4D77C
:10BCCC001200E80E026E030E036EEDDF042EF9D7A0
:10BCDC00120030C0EAFF2FC0E9FFEFCF26F0265349
:10BCEC00D8B413D02D6B010E265DD8A00ED02D2B01
:10BCFC002D512F25E96EE86A3021EA6EEFCF27F03F
:10BD0C000FD826512D5DD8A0F2D712009EAAFED7CF
:10BD1C009EBAAECF27F0ABA202D0AB98AB88120084
:10BD2C009EA8FED727C0ADFF1200700ED312E06A9A
:10BD3C00F86AC290C09EC186C184C182C180070EC0
:10BD4C00B46E806A816A826A846A1200400EAF6E99
:10BD5C00030EB06EB886AC84AC98AB8EAB88AC8A54
:10BD6C001200006809500562006A1200006A09504E
:10BD7C00056212000A500662120000681200006888
:10BD8C0009500560006A1200006A06500A5CD8A0CF
:10BD9C0012000A50065C04E30950055CD8B012008E
:10BDAC0000681200006A016A080E046ED89005360D
:10BDBC0000360950005E0580D8B003D005900950BC
:10BDCC000026042EF3D7120006C008F005C007F0B9
:10BDDC000AC00CF009C00BF0026A036A0CC006F032
:10BDEC000BC005F0096A0A6AC1DF00A003D0056A1E
:10BDFC00066A1200100E046ED8900736083602360A
:10BE0C0003360B50025E0C50035A0780D8B005D095
:10BE1C0007900B5002260C500322042EEDD708C0BD
:10BE2C0006F007C005F003C001F002C000F01200DC
:10BE3C0005500902F3CF00F0F4CF01F005500A02CF
:10BE4C00F350012606500902F350012606520A024D
:10BE5C0012000900F5CF05F0F5CFE7FF090005D07A
:10BE6C000900F550056E062609000552D8B41200DB
:10BE7C000900F5CFE4FF052EFBD712002727436FEF
:10BE8C006E666967203D2033326D687A204D434CD5
:10BE9C005220424F44454E20494E54494F37204C76
:10BEAC0045443D42330026263D3D3D20546572728B
:10BEBC0079277320426F6F746C6F61646572203DDB
:10BECC003D3D2020763920392F32302F31351B1B48
:10BEDC0053656E6420686578206F7220707265738C
:10BEEC0073205820746F20657869740002023E201C
:10BEFC000B0B496E76616C696420686578000D0DDA
:10BF0C00496E76616C696420636F756E74000E0EF9
:10BF1C00436865636B73756D206572726F720E0E7C
:10BF2C00496E76616C6964207265636F726412127B
:10BF3C0053656E642045534320666F72206D656EA9
:10BF4C00752001012E001010496E76616C69642019
:10BF5C0061646472657373200D0D20455343207426
:08BF6C006F207265736574001B
:020000040030CA
:06000100090F1EFF8381C0
:0600080007C007E00740FD
:00000001FF
